:020000040000FA
:0400000009303A2861
:08000800A000030EA100831209
:100010008B1C32288B1031181428B11C3228643004
:10002000010203183128182800001628172818285C
:1000300019281A281B281C281D281E281F283110A3
:10004000B114A810031005190314AA0DA90DA80DC9
:10005000B00B322831152A08AF002908AE00280855
:10006000AD00B11081010B11210E8300A00E200EF6
:02007000090085
:0C007400203084008001840A6030040207
:10008000031C3C281230B0006F218316FF23900020
:10009000831283160C308505870183128501870141
:1000A000073099000030831691009F008312C830FA
:1000B00083168100831231309000003083168C004B
:1000C000831210308B00831600309B001C141A081A
:1000D0008312BC00831610309B001C141A08831274
:1000E000BD008F2181018E018F010B118B100B1030
:1000F0008C018B17892031199F20B30B872803109F
:1001000085190314B90DF030390203190221982121
:100110007A286400311808000B1D08000B11B1107B
:1001200031141230B000051D9A28321483160113C1
:100130008312080032108316011783120800311150
:100140000130B7008B132030370783169B001C1437
:100150001A088312A400A500C030A5061030370786
:1001600083169B001C141A088312A3000030370763
:1001700083169B001C141A088312A2008B17321CD2
:10018000C72822090339A200A309A409A509220846
:100190002D02031DFC2823082E02031DFC28240821
:1001A0002F02031DE52801303702031DDC283D180E
:1001B000DC283D143E14722102303702031DE5286D
:1001C000BD18E528BD143E147D2125082F02031D0E
:1001D000FC2801303702031DF2283D1CF2283D1097
:1001E0003E14802102303702031DFB28BD1CFB2872
:1001F000BD103E148221FC28B70A033037020318D1
:100200000800A2280130B600B300B400B500B70062
:1002100085018701B1138920B30B222903108519A9
:100220000314B90DF030390203194929B40B2229FE
:100230000130370203198521023037020319892161
:100240009630B400311D0B293111321C2C292D0997
:100250000339AD00AE09AF092F1CB1132F1C0B29B8
:10026000B11B0B292E180B29B1178B132030370720
:10027000BB002F08BA005C2110303707BB002E08E6
:10028000BA005C2100303707BB002D08BA005C21A2
:100290008B1785018701B70AB60103303702031CAB
:1002A0000B298F2108003E1C08003E101030BB00B7
:1002B0003D08BA005C2108008B133A0883161C1510
:1002C0009A003B089B0055309D00AA309D009C146D
:1002D00064009C1868291C1183128B170800FF30DA
:1002E000C300080041101E304005031D0800C01463
:1002F000C01A0800FF30C3000800851285140800EA
:10030000411408008516851008000508113A85007B
:1003100008000508223A8500080008000800C0010E
:10032000C1013D18C014BD188514BD1C85160800F8
:100330008F08031908008F01C30FA629C30A0310F1
:10034000C00D4118A629C01AC015C012FC22C20057
:1003500068304005031D0510401334304005031D6F
:10036000051242080E020318BD2914304005031D72
:10037000051408304005031D05168F08031D0800ED
:10038000640042080E02031CBD2914304005031D01
:10039000051028304005031D05142C304005031DB1
:1003A000051210304005031D051601304302031DE0
:0603B000080053210800C3
:0805F80003308A00430382076F
:100600000034043407340B340F34123416341934E4
:100610001C3420342334263429342C342F343334FE
:10062000363438343B343E3441344434473449342E
:100630004C344F3451345434563459345B345E3472
:10064000603462346534673469346C346E347034C9
:1006500072347434763478347A347C347E34803432
:10066000823484348634883489348B348D348F34A6
:100670009034923494349534973498349A349B342B
:100680009D349E34A034A134A334A434A634A734BA
:10069000A834AA34AB34AC34AE34AF34B034B13453
:1006A000B234B434B534B634B734B834B934BA34F7
:1006B000BB34BD34BE34BF34C034C134C234C3349F
:1006C000C434C434C534C634C734C834C934CA3455
:1006D000CB34CC34CC34CD34CE34CF34D034D0340D
:1006E000D134D234D334D334D434D534D534D634CD
:1006F000D734D734D834D934D934DA34DB34DB3492
:10070000DC34DD34DD34DE34DE34DF34DF34E03459
:10071000E034E134E234E234E334E334E434E43426
:10072000E534E534E534E634E634E734E734E834F8
:10073000E834E934E934E934EA34EA34EB34EB34CC
:10074000EB34EC34EC34EC34ED34ED34EE34EE34A4
:10075000EE34EF34EF34EF34F034F034F034F0347E
:10076000F134F134F134F234F234F234F334F3345A
:10077000F334F334F434F434F434F434F534F53439
:10078000F534F534F634F634F634F634F734F73419
:10079000F734F734F734F834F834F834F834F834FC
:1007A000F934F934F934F934F934FA34FA34FA34DE
:1007B000FA34FA34FA34FB34FB34FB34FB34FB34C4
:1007C000FB34FB34FC34FC34FC34FC34FC34FC34AB
:1007D000FC34FD34FD34FD34FD34FD34FD34FD3492
:1007E000FE34FE34FE34FE34FE34FE34FE34FE3479
:0E07F000FE34FF34FF34FF34FF34FF34FF3497
:084000000B000300040008009E
:02400E00CC01E3
:10420000010003000300030003000200020002009B
:1042100002000000000000000000FF00FF00FF009F
:10422000000000000000000000000000000000008E
:104230000000C000C000C000C000FF00FF00FF0081
:104240000100C300F300CF00FF00C300F300CF0064
:10425000FF00C300F300CF00FF00FF00FF00FF00DE
:10426000FF00FF00FF00FF00FF00FF00FF00FF0056
:10427000FF00FF00FF00FF00FF00FF00FF00FF0046
:10428000FF00FF00FF00FF00FF00FF00FF00FF0036
:10429000FF00FF00FF00FF00FF00FF00FF00FF0026
:1042A000FF00FF00FF00FF00FF00FF00FF00FF0016
:1042B000FF00FF00FF00FF00FF00FF00FF00FF0006
:1042C000FF00FF00FF00FF00FF00FF00FF00FF00F6
:1042D000FF00FF00FF00FF00FF00FF00FF00FF00E6
:1042E000FF00FF00FF00FF00FF00FF00FF00FF00D6
:1042F000FF00FF00FF00FF00FF00FF00FF00AA001B
:00000001FF
